:10F800000C94387C0C94537C0C94537C0C94537C57
:10F810000C94537C0C94537C0C94537C0C94537C2C
:10F820000C94537C0C94537C0C94537C0C94537C1C
:10F830000C94537C0C94537C0C94537C0C94537C0C
:10F840000C94537C0C94537C0C94537C0C94537CFC
:10F850000C94537C0C94537C0C94537C0C94537CEC
:10F860000C94537C0C94537C0C94537C0C94537CDC
:10F8700011241FBECFEFD0E1DEBFCDBF11E0A0E06D
:10F88000B1E0E4E5FFEF02C005900D92A430B107AE
:10F89000D9F712E0A4E0B1E001C01D92A634B1078F
:10F8A000E1F70C946C7F0C94007C0F92AF93BF93A4
:10F8B000CF93DF93EF93FF93FC01EA01DB01C8953F
:10F8C000099231961197D9F7FF91EF91DF91CF917E
:10F8D000BF91AF910F9008950F921F920F93AF9326
:10F8E000BF93CF93DF93EF93FF93FC01EA01DB011A
:10F8F0000990199001E043D032961297C9F7FC01A4
:10F9000003E03DD005E03BD0FF91EF91DF91CF9137
:10F91000BF91AF910F911F900F9008950F931F9378
:10F92000EF93FF93FC0103E02AD000E011E0E00F29
:10F93000F11FE617F707B9F7FF91EF911F910F91AC
:10F9400008950F930F9222D0082E09E018D00F903F
:10F950000F9108950F930F92EF93FF9317D0FC012F
:10F9600060935700C895802DFF91EF910F900F91F4
:10F9700008950F930BD001E102D00F910895F999EA
:10F98000FECF00935700E895FFFF0000009157005D
:10F9900000FDFCCF089589E08093C4008091C100F0
:10F9A00088618093C10008958091C100877E809313
:10F9B000C10008958093C6008091C00086FFFCCFEF
:10F9C0008091C00080648093C00008958091C6003B
:10F9D000992708958091C0009927807890700895A4
:10F9E000EF92FF920F931F93CF93DF937B01C0E0C1
:10F9F000D0E0C617D70770F48C010E94EA7C8823F8
:10FA0000E1F30E94E67CF80181938F012196CE15E7
:10FA1000DF0598F381E090E0DF91CF911F910F9186
:10FA2000FF90EF900895EF92FF920F931F93CF9363
:10FA3000DF937C018B01C0E0D0E0C017D10738F420
:10FA4000F70181917F010E94DA7C2196F6CF81E057
:10FA500090E0DF91CF911F910F91FF90EF9008956B
:10FA6000EF92FF920F931F93CF93DF937C0100E0FF
:10FA700010E00817190788F4C0E0D0E000000E94E9
:10FA8000EA7C882351F4219688E0CA3CD807B0F379
:10FA90000F5F1F4F0E151F0578F3DF91CF911F9158
:10FAA0000F91FF90EF9008950E94D47C0E94000077
:10FAB0000895DF92EF92FF920F931F93CF93DF93FE
:10FAC000CDB7DEB72197DEBFCDBF8C017B01198298
:10FAD000D98061E070E0CE01860F971F0E94F07C14
:10FAE00089818B31B1F761E070E0C8010E94F07C40
:10FAF00061E070E0CE01860F971F0E94F07C898143
:10FB00009927182F002761E070E0CE01860F971F1C
:10FB10000E94F07C8981080F111D61E070E0CE0128
:10FB2000860F971F0E94F07C89818E30B9F4C8013E
:10FB30000196BC01C7010E94F07C98018FEF0F3F36
:10FB4000180779F0F70181917F01D82621503040C4
:10FB5000FFEF2F3F3F07B1F7DD2019F080E090E085
:10FB600001C0C8012196DEBFCDBFDF91CF911F91AB
:10FB70000F91FF90EF90DF900895CF92DF92FF9268
:10FB80000F931F93CF93DF93182FEB016A018BE143
:10FB90000E94DA7C4BE1F42E812F0E94DA7CF12660
:10FBA0000D2F1127802F0E94DA7CF0268C2F0E94C7
:10FBB000DA7CFC268EE00E94DA7C8EE0F826219723
:10FBC0008FEFCF3FD80759F0F60181916F01F826EA
:10FBD0000E94DA7C2197FFEFCF3FDF07A9F78F2D37
:10FBE0000E94DA7CDF91CF911F910F91FF90DF90FF
:10FBF000CF90089599278139910559F0823991055F
:10FC000024F48039910529F008C08239910519F052
:10FC100004C082E003C087E001C080EC992708950A
:10FC2000BF92CF92DF92EF92FF920F931F93CF93E9
:10FC3000DF93B82E8B01FB018081C82FDD27C231F5
:10FC4000D10509F46DC0C331D105DCF4C330D10551
:10FC500009F44DC0C430D10544F4C130D10579F167
:10FC6000C230D10509F44AC003C1C630D10509F438
:10FC70004AC0C630D1050CF4FBC060970CF4F8C044
:10FC800054C0C531D10509F4C7C0C631D10544F40B
:10FC9000C331D10509F471C0649709F449C0E8C0C3
:10FCA000CA31D10509F4D6C0CB31D10524F4669709
:10FCB00009F499C0DDC06B9709F4C3C0D9C0FB013A
:10FCC000118288E0828381E4838386E5848382E5F0
:10FCD000858389E4868383E5878380E580878FE554
:10FCE000818782E38287AB016BE070E0C7C0FB01D4
:10FCF00081810E94FA7DF801828301C0FB0111829B
:10FD0000A801BE01BBC0FB0183819927982F8827DA
:10FD10002481820F911D909345028093440206C076
:10FD200060E070E0CB010E948E7CF8011182A3C0DC
:10FD3000FB0181819927D82FCC2782819927C82B55
:10FD4000D92B1182CB0102962091440230914502B9
:10FD5000AC01BE01C901880F991F0E94557CF801B2
:10FD6000EC0FFD1F12829E0136952795809144026B
:10FD700090914502820F931F49C0FB018181992711
:10FD8000D82FCC2782819927C82BD92BCC24DD24CE
:10FD9000CC16DD06D8F4FAE0EF2EF12CE60EF71EB5
:10FDA0008091440290914502880F991FA70160E05D
:10FDB00071E08C0D9D1D0E946C7C80E091E0C80E6E
:10FDC000D91EE80EF91ECC16DD0650F30E94B97C50
:10FDD000F8011182D695C795809144029091450211
:10FDE0008C0F9D1F29C0FB0181819927D82FCC271B
:10FDF00082819927C82BD92B1182EC0FFD1F12820B
:10FE000080914402909145028C0F9D1F9093450272
:10FE100080934402239674CFFB0181819927382F68
:10FE2000222782819927282B392B11828091440225
:10FE300090914502820F931F909345028093440254
:10FE40001AC0FB0111828481E82FFF27E050FF4F89
:10FE5000808107C0FB01118269E081E090E00E948F
:10FE6000AA7CF80182831382A80164E070E006C0D6
:10FE700089ECF8018183A80162E070E08B2D0E947B
:10FE8000BD7DDF91CF911F910F91FF90EF90DF909B
:10FE9000CF90BF900895CF93DF93CDB7DEB7219772
:10FEA000DEBFCDBF69E081E090E00E94AA7C992787
:10FEB00084FF09C08F7E0E94A17C05C064E071E0D0
:10FEC00089810E94107E64E071E0CE0101960E945B
:10FED000597D892B99F3F7CFCFEFD0E1DEBFCDBFAE
:10FEE000CEE1F894AEEFB7E00E94A17F802D843B75
:10FEF00079F4AFEFB7E00E94A17F802D833C41F4FD
:10FF0000ADEFB7E00E94A17F802D99278093660016
:10FF10000E94CB7C0E94E67C84E690E00E94307DCB
:10FF20000E94EA7C882319F00E944B7F04C0C150D4
:10FF3000C5B9CC2389F70E94547D80E090E00C94F1
:10FF4000A97FF999FECFB2BDA1BDF89A119600B470
:04FF50000895FFCF42
:04FF54001E960900EC
:040000030000F80001
:00000001FF
